:0800000000008A110A12052814
:06000A003830FE00013059
:10001000FF0080308A110A120C218A110A12831201
:100020000313AD007F08AC003A30AE000130AF00E2
:10003000831203132C08B0002D08B100FF30AC0769
:10004000031CAD03300831040319952804302E0732
:10005000B000B101B10D2F08B1073008FE00310822
:10006000FF0080308A110A120C218A110A128312B1
:100070000313B3007F08B2002E08FE002F08FF0014
:1000800080308A110A120C218A110A12831203137A
:10009000B500B1007F08B400B00002302E07B000F8
:1000A000B101B10D2F08B1073008FE003108FF0083
:1000B00080308A110A120C218A110A12831203134A
:1000C000B100B7007F08B000B600831203133208F6
:1000D000B6003308B700FF30B207031CB30336087D
:1000E000370403198E283408FE003508FF008030DD
:1000F0008A110A12F9208A110A1283120313B60018
:100100003008840083133118831736088000B40A3E
:100110000319B50AB00A0319B10A6528063083121B
:100120000313AE070318AF0A18288A110A12992878
:100130000800EB20013083120313AA002D30A90020
:100140008030AB002908FE002A08FF002B08AB20F6
:10015000E5209A28080083120313A3007F08A20059
:100160007E08A100A4018312031324082107A5001F
:1001700022080318013EA60023080318013EA70029
:100180002508FE002608FF0027088A110A12F92018
:100190008A110A1283120313A80028080319D6280B
:1001A0002808D72083120313A40AB3280800831257
:1001B0000313A000831203130C1EDA288312031307
:1001C00020088312031399000800831203138C1E66
:1001D000E5281A08080083160313181581309900C2
:1001E0001812831203139817181683160313981600
:1001F0000800003A03190029803A0319072900343E
:100200007E08840083137F188317000808007F0886
:100210008A007E0882000800003A03191429803AF7
:1002200003191E29FF0100347E08840083137F1800
:1002300083170008FF00840A000808008A110A12C8
:100240000721FD00FE0FFF03FF0A8A110A12072192
:10025000FC007D08FF007C08080050346F346434D3
:1002600065346D346F3473342134213421340034D7
:100270000134003440340134383400340134003463
:02028000003448
:00000001FF
